:100000005FEF27F00000000000EF00F000000000AC
:100010000000000000000000F3D7FFFF0201F251D2
:10002000000A32E0016A015007081CE303016FBFB8
:1000300002D0939E01D0938E060E0D6E0D2EFED72C
:100040000000938C060E0D6E0D2EFED70000939CC3
:10005000060E0D6E03010D2EFDD700006F376F9158
:10006000012AE1D7938E060E0D6E0D2EFED70000ED
:10007000938C060E0D6E0D2EFED70000939C060E7F
:100080000D6E0D2EFED7000012000201F251000A83
:1000900018E0938C060E0D6E0D2EFED70000938E89
:1000A000060E0D6E0D2EFED70000939E060E0D6EF1
:1000B0000D2EFED70000939C060E0D6E0D2EFED762
:1000C00000001200086A096A100E0C6E013408362E
:1000D00009360450085E0550D8A0053C095ED8B02A
:1000E00007D0045008260550D8B0053C0926D89002
:1000F000003601360C2EEAD712000AAE029E000E20
:1001000012000201FC5103016B256E6FBEDFF2C2CB
:100110006FF384DF03016F6B81DF03016A51B00F5E
:100120006F6F7CDF03016E510F0804E36EC36CF345
:100130006D6B19D06EC302F00232029E0232029E33
:100140000232029E0232029E02C06DF302C000F033
:100150000036009000360090003600900036009087
:1001600000506E5D6C6F6CC36FF358DF03016D510F
:10017000100F6F6F53DF89DFF2C26FF34FDF400E56
:1001800003016F6F4BDF12000201F251000A12E00F
:10019000939E060E0D6E0D2EFED70000938C060E5C
:1001A0000D6E0D2EFED70000938E060E0D6E0D2ED9
:1001B000FED7000012000B840BAEE6EF00F0010E3C
:1001C000036E026A016A006A0A360232FF0E1200EA
:1001D000220E0C6E086A096A0A6A0B6A0C06D8B409
:1001E0001FD0D8900B320A32093208320332023261
:1001F00001320032D8A0F2D70C06D8B409D004508E
:1002000008260550092206500A2207500B22EAD779
:10021000045008260550092206500A2207500B22D6
:100220001200026A016A006A086A036A000E12007C
:10023000A00E0301626F0F0E636F000E646F656F97
:10024000A00E006E0F0E016E000E026E000E036E09
:1002500060C304F061C305F0000E066E076EB8DFE0
:1002600000C062F301C063F302C064F303C065F32E
:10027000000E035C08E1000E025C05E1020E015C69
:1002800002E1940E005C01E231D0940E625F020E36
:10029000635B000E645B655B050E006E005007E05B
:1002A0006533643363336233659FFF0FF8D762C3EE
:1002B00000F063C301F064C302F065C303F0010EF4
:1002C000625F000E635B645B655B005001100210AF
:1002D00003100CE00000000000000000000000001F
:1002E00000000000000000000000E1D712000B80B9
:1002F0000BAE83EF01F0026A0AAEFF0E026E016ED2
:10030000006E0A360232FF0E12000301646B050E06
:10031000645D0AE264516225E16E000E6321E26EC3
:10032000200EE66E642BF3D764516225E16E000E59
:100330006321E26EE66A640764516225656F000E10
:100340006321666F0A0E046E000E056E60C300F036
:1003500061C301F0B7DE08C000F009C001F0300E43
:10036000002665C3E1FF66C3E2FF00C0E6FF0A0E98
:10037000046E000E056E60C300F061C301F0A2DEE2
:1003800000C060F301C061F3000E011802E1000E2D
:10039000001801E102D06407CFD7120076DEF2C266
:1003A0006FF33CDE400E03016F6F38DE61C36AF30A
:1003B00060C36BF3A6DE0301656B6451655DD8B065
:1003C000B3D065516225E96E000E6321EA6EEE50EE
:1003D000000A02E1676B09D065516225E96E000EE3
:1003E0006321EA6E200EEE5C676F666B665104084F
:1003F000D8A092D0050E6703F3CF00F0F4CF01F040
:1004000066510026000E01223D0E0024F66E540EA9
:100410000120F76E000EF86E000E01BEFF0EF822EE
:100420000900F5CF68F36151020A000ED8A4010E4D
:10043000016E6151040A000ED8A4010E006E005036
:1004400001166151060A000ED8A4010E006E01507B
:10045000001629E068B702D0699F01D0698F68B79C
:1004600002D0699D01D0698D68B502D0699B01D029
:10047000698B68B502D0699901D0698968B302D0E7
:10048000699701D0698768B302D0699501D0698501
:1004900068B102D0699301D0698368B102D06991D3
:1004A00001D0698120D068B502D0699F01D0698FE1
:1004B00068B502D0699D01D0698D68B302D0699B8F
:1004C00001D0698B68B302D0699901D0698968B19C
:1004D00002D0699701D0698768B102D0699501D0CF
:1004E00069856993699169C36FF398DD0201FA51D7
:1004F000040A010ED8A4000E016EFA51050A010E7D
:10050000D8A4000E006E0150001203E069C36FF31F
:1005100085DD0301662B6AD76F6B80DD03016F6B8E
:100520007DDD0301652B49D76151010F6A6F60C3FF
:100530006BF3E7DD0301656B6451655DD8B0BBD03B
:1005400065516225E96E000E6321EA6EEE50000AE5
:1005500002E1676B09D065516225E96E000E6321E7
:10056000EA6E200EEE5C676F666B66510408D8A0D9
:100570009AD0050E6703F3CF00F0F4CF01F0665177
:100580000026000E01223D0E0024F66E540E0120BE
:10059000F76E000EF86E000E01BEFF0EF822090085
:1005A000F5CF68F36151020A000ED8A4010E016E66
:1005B0006151040A000ED8A4010E006E005001160D
:1005C0006151060A000ED8A4010E006E01500016FB
:1005D00029E068BF02D0699F01D0698F68BF02D04F
:1005E000699D01D0698D68BD02D0699B01D0698B7E
:1005F00068BD02D0699901D0698968BB02D069974A
:1006000001D0698768BB02D0699501D0698568B956
:1006100002D0699301D0698368B902D0699101D091
:10062000698128D068BD02D0699F01D0698F68BDFB
:1006300002D0699D01D0698D68BB02D0699B01D051
:10064000698B68BB02D0699901D0698968B902D009
:10065000699701D0698768B902D0699501D0698529
:1006600068B702D0699301D0698368B702D06991F5
:1006700001D0698169C36FF3D1DC0201FA51040A28
:10068000010ED8A4000E016EFA51050A010ED8A47D
:10069000000E006E0150001203E069C36FF3BEDC70
:1006A0000301662B62D76F6BB9DC03016F6BB6DC9D
:1006B0000301652B41D768DD12000B820BAE67EF9B
:1006C00003F003680268016800680A360232FF0E10
:1006D00012000C6A0E6A0250D8A482EF03F001C027
:1006E00002F000C001F0006A0E860250D8A482EF2A
:1006F00003F001C002F0016A0E960E880250D8B4D1
:1007000094EF03F00E50035ED8A4D8A099EF03F045
:10071000D89002BE9EEF03F0003601360236032E5B
:1007200089EF03F099EF03F0010E0C6E7ADDA1EF73
:1007300003F0020E0C6E3FDDA1EF03F0040E0C6E11
:10074000DCDC12001D0E0D6E0D2EFED71200030113
:10075000616B0201F36B010EF96F60C361F303017A
:100760006137619161376191613761916137619161
:100770000201F45303E0080E030161270201F9535B
:1007800003E0040E030161270201F35303E0020EAC
:10079000030161270201FD5302E00301612B75DCB7
:1007A000F2C26FF33BDC61C36FF338DCEDDC060EA5
:1007B0000C6E300E0D6E0D2EFED70C2EFCD70000E9
:1007C000040E0301615F61DCF2C26FF327DC61C3D9
:1007D0006FF324DCD9DC060E0C6E300E0D6E0D2E80
:1007E000FED70C2EFCD7000012000B6A0A6A096AB9
:1007F00000500402F4CF09F0F3CF08F001500502D5
:10080000F4CF0BF0F3CF0AF000500502F3500926A5
:10081000F4500A22E86A0B2201500402F350092620
:10082000F4500A22E86A0B2208C000F009C001F067
:100830000AC002F00BC003F012000201E451000AEA
:1008400025E1030156B102D08A9601D08A8656B3BB
:1008500002D0899401D0898456B502D08A9801D0FB
:100860008A8856B702D0899601D0898656B902D0B7
:100870008A9A01D08A8A56BB02D0899A01D0898A85
:1008800056BD02D0899801D0898824D0030156B181
:1008900002D08A8601D08A9656B302D0898401D0CC
:1008A000899456B502D08A8801D08A9856B702D06A
:1008B000898601D0899656B902D08A8A01D08A9A4F
:1008C00056BB02D0898A01D0899A56BD02D0898848
:1008D00001D0899805C360F306C361F3A9DC120057
:1008E0000B6A0B86FF0E12000CB0B6EF04F00CA2E0
:1008F0005EEF05F00E6A000E0264CDEF04F0F00E1C
:100900000214D8A498EF04F0023A01380F0B022623
:100910000138F00B016E00380F0B01260038F00B88
:10092000006E08380F0B00260838F00B086E0E8496
:10093000D89002BEB1EF04F0083600360136023618
:100940000E2A02BEB1EF04F0083600360136023638
:100950000E2A02BEB1EF04F0083600360136023628
:100960000E2A0E50036452EF05F0035E0BBC08AE76
:1009700058EF05F0D880800E08640030000E002289
:1009800001220222D8A058EF05F0023201320032D3
:10099000034A5EEF05F058EF05F001C002F000C019
:1009A00001F008C000F0086A000E0E86026404EF31
:1009B00005F0F00E0214D8A4ECEF04F0023A01386E
:1009C0000F0B02260138F00B016E00380F0B0126C9
:1009D0000038F00B006E0E84D89002BEB1EF04F028
:1009E0000036013602360E2A02BEB1EF04F00036A0
:1009F000013602360E2A02BEB1EF04F0003601368F
:100A000002360E2AB1EF04F001C002F000C001F07E
:100A1000006A000E0E960E88026431EF05F0F00EAB
:100A20000214D8A41CEF05F0023A01380F0B02267D
:100A30000138F00B016E0E84D89002BEB1EF04F0C5
:100A4000013602360E2A02BEB1EF04F0013602363C
:100A50000E2A02BEB1EF04F0013602360E2AB1EFC3
:100A600004F001C002F0016A000E0E86026463EF1A
:100A700005F0F00E0214D8A440EF05F0023A0E84FF
:100A8000D89002BEB1EF04F002360E2A02BEB1EFDA
:100A900004F002360E2A02BEB1EF04F002360E2A2E
:100AA000B1EF04F0010E0C6EDBEC00F067EF05F027
:100AB000020E0C6E7DEC00F067EF05F0040E0C6E7C
:100AC000FCDD67EF05F0080E0C6E11EC01F0120072
:100AD0000450085E0550D8A0053C095E0650D8A019
:100AE000063C0A5E0750D8A0073C0B5E0336070E93
:100AF0000C6E0334083609360A360B36045003A050
:100B00000ED0085E0550D8A0053C095E0650D8A05E
:100B1000063C0A5E0750D8A0073C0B5E0DD00826A5
:100B20000550D8B0053C09260650D8B0063C0A2628
:100B30000750D8B0073C0B2603360C2EDAD7023408
:100B4000083609360A360B36045003A00ED0085E6C
:100B50000550D8A0053C095E0650D8A0063C0A5EA8
:100B60000750D8A0073C0B5E0DD008260550D8B022
:100B7000053C09260650D8B0063C0A260750D8B0D6
:100B8000073C0B260236070E0C6E02340836093677
:100B90000A360B36045002A00ED0085E0550D8A0CD
:100BA000053C095E0650D8A0063C0A5E0750D8A056
:100BB000073C0B5E0DD008260550D8B0053C092631
:100BC0000650D8B0063C0A260750D8B0073C0B2682
:100BD00002360C2EDAD70134083609360A360B36BF
:100BE000045002A00ED0085E0550D8A0053C095E56
:100BF0000650D8A0063C0A5E0750D8A0073C0B5E02
:100C00000DD008260550D8B0053C09260650D8B0AE
:100C1000063C0A260750D8B0073C0B260136070EC3
:100C20000C6E0134083609360A360B36045001A022
:100C30000ED0085E0550D8A0053C095E0650D8A02D
:100C4000063C0A5E0750D8A0073C0B5E0DD0082674
:100C50000550D8B0053C09260650D8B0063C0A26F7
:100C60000750D8B0073C0B2601360C2EDAD70034DB
:100C7000083609360A360B36045001A00ED0085E3D
:100C80000550D8A0053C095E0650D8A0063C0A5E77
:100C90000750D8A0073C0B5E0DD008260550D8B0F1
:100CA000053C09260650D8B0063C0A260750D8B0A5
:100CB000073C0B260036070E0C6E0034083609364A
:100CC0000A360B36045000A00ED0085E0550D8A09E
:100CD000053C095E0650D8A0063C0A5E0750D8A025
:100CE000073C0B5E0DD008260550D8B0053C092600
:100CF0000650D8B0063C0A260750D8B0073C0B2651
:100D000000360C2EDAD700B00ED00450082605505D
:100D1000D8B0053C09260650D8B0063C0A26075034
:100D2000D8B0073C0B2612000B1E0A1E091E081E17
:100D3000082AD8B4092AD8B40A2AD8B40B2A12002F
:100D4000830EC21656C300F00036009000360090A5
:100D50000050C212F7DCC282C2A201D0FDD7C4CFBC
:100D600001F0006AC3500012000E011212000301CC
:100D70005C6B5D6B56C35EF357C35FF3800E571910
:100D8000006E800E005C02E1000E565D0BE2010E6B
:100D90005C6F000E5D6F565100085E6F57C35FF3C6
:100DA000000E5F575EC360F35FC361F358C362F325
:100DB00059C363F385EC01F0060E5A6F000E5B6FAA
:100DC000000E006E5B51005C02E15A51000819E20E
:100DD0005A515825E16E5B515921E26E010E5A5D60
:100DE000006E000E5B59016E00505825E96E0150EF
:100DF0005921EA6EEECFE6FF010E5A5F000E5B5BF3
:100E0000DFD758C3E1FF59C3E2FF200EE66E5C5105
:100E10005D111AE05A6B5B6B5A515825E96E5B51B4
:100E20005921EA6EEE50200A03E15A4B5B2BF4D7AE
:100E3000010E5A5F000E5B5B5A515825E16E5B5103
:100E40005921E26E2D0EE66E12000B6A0350D8B4E3
:100E50006BEF07F002500A6E028E8E0E035E03AE39
:100E60006FEF07F0036C080E035CD8A04AEF07F0A1
:100E7000036E013602C001F0026A080E035CD8A0BE
:100E80004AEF07F0036E0136016A0350D8A4D890E8
:100E900054EF07F00350D8B454EF07F0D890023263
:100EA0000132032E4EEF07F00BBC01A061EF07F0FB
:100EB000D8A061EF07F0012AD8B4022A02BE7EEF63
:100EC00007F00AAE84EF07F0021E011E012AD8B413
:100ED000022A84EF07F0026A016A84EF07F00B80B0
:100EE0000BAE88EF07F0026A0AAE88EF07F0FF0E3C
:100EF000026E016E0A36023288EF07F0010E0C6EA8
:100F000077EC01F08AEF07F0000E0C6E8AEF07F025
:100F1000FF0E0C6E0150006E0250016E1200005068
:100F2000086E0150006E016A026A036A0B6A0C6A5D
:100F3000960E036E0A6A00C001F008C000F0086A4D
:100F4000026A69EC03F01200030156B102D08B9ED5
:100F500001D08B8E56B302D08B9601D08B8656B5BE
:100F600002D08B9C01D08B8C56B702D08B9401D0D1
:100F70008B8456B902D08B9A01D08B8A56BB02D093
:100F80008B9201D08B8256BD02D08B9801D08B887A
:100F900005C360F306C361F318EC01F0120002010F
:100FA000FA51040A010ED8A4000E016EFA51050A86
:100FB000010ED8A4000E006E015000120DE057C3C0
:100FC00060F356C361F358C362F359C363F35AC362
:100FD00064F3CEEC01F05DD0FA51020A010ED8A400
:100FE000000E016EFA51030A010ED8A4000E006E25
:100FF0000150001214E0070E03015703F3CF60F312
:10100000040E602756C361F36137619158C362F3E0
:1010100059C363F35AC364F3CEEC01F03AD0FD6BCD
:1010200056C300F000360090003600900050080FC4
:101030000301606FA7EC03F057C360F3A7EC03F064
:10104000010EFD6F03015B6B5A515B5D22E25B5148
:101050005825E96E000E5921EA6EEECF01F001C06D
:1010600060F36033609F6033609F6033609F6033E4
:10107000609FA7EC03F003015B515825E96E000E59
:101080005921EA6EEECF60F3A7EC03F003015B2B6E
:10109000DBD71200086A096A000E07620364CFEF0B
:1010A00008F0025006180A6E075003267E0ED8A0DC
:1010B00060EF08F0035ED8B0D4EF08F064EF08F0FA
:1010C000035ED8A0D9EF08F0028E068E02C00EF0A3
:1010D00001C00BF000C00DF000500402F4CF0CF082
:1010E00001500502F4CF00F0F3CF08F00402F350F2
:1010F0000C26F4500822000E00220D500502F35079
:101100000C26F4500822000E002202500402F35074
:101110000826F450002202500502016A000E012246
:10112000F3500026F45001220D500602F350082619
:10113000F4500022026A000E012202220B50060225
:10114000F3500026F4500122000E02220E50060237
:10115000F3500126F450022202BEB7EF08F0083621
:101160000036013602360306D8B4D9EF08F0CAEFCC
:1011700008F0D880800E08640030000E00220122A2
:101180000222D8A0CAEF08F0023201320032034A2C
:10119000D4EF08F00AAE029E000EDCEF08F0010E5C
:1011A00011EC01F0DCEF08F0020E5DEC03F0DCEF77
:1011B00008F0040EDBEC00F012000450000A12E10B
:1011C0000550000A0FE10650000A0CE10750000A22
:1011D00009E1FF0E006EFF0E016EFF0E026E7F0E24
:1011E000036E97D00C6A07BE0C2A0D6A0B6A0A6A56
:1011F000096A086A0350021001100010D8B484D0A4
:10120000035007180E6E0EBE0D1E07AE0BD0041E47
:10121000051E061E071E042AD8B4052AD8B4062ABD
:10122000D8B4072A03AE0BD0001E011E021E031EF7
:10123000002AD8B4012AD8B4022AD8B4032A035009
:1012400007100E6E0EBE1CD043DC0CBE36D00DAEA9
:101250005BD0001E011E021E031E002AD8B4012A04
:10126000D8B4022AD8B4032A081E091E0A1E0B1E6F
:10127000082AD8B4092AD8B40A2AD8B40B2A44D0E8
:1012800007AE15D003BE0DD003500B6E02500A6E90
:101290000150096E0050086E036A026A016A006A12
:1012A000D6D7036A026A016A006A002A000C031E8C
:1012B000021E011E001E0C8EC7D7082AD8B4092AA8
:1012C000D8B40A2AD8B40B2A0450085CD8A4BFD7D3
:1012D0000550095CD8A4BBD706500A5CD8A4B7D780
:1012E00007500B5CD8A4B3D70B6A0A6A096A086A6C
:1012F000002AD8B4012AD8B4022AD8B4032A03AEEB
:10130000A6D70E6A0E88FF0C0E6A0CA001D00CDD69
:10131000000F12000450000A12E10550000A0FE10C
:101320000650000A0CE10750000A09E1FF0E006EAA
:10133000FF0E016E7F0E026EFF0E036EA8D0086ACC
:10134000096A0750D8B435EF0AF00350D8B43AEF21
:101350000AF0025006180A6E028E068E0E6A02C04D
:1013600008F001C00CF000C00DF004500D5E0550F7
:10137000D8A0053C0C5E0650D8A0063C085E086A62
:101380000C6A0D6AD8A0CCEF09F0D8900232013275
:1013900000320832010E0E6E0750035ED8A0D9EF5E
:1013A00009F07E0E0E240326D8B03FEF0AF0DFEFDF
:1013B00009F07E0E0E240326D8A044EF0AF0180E82
:1013C0000B6E0D360C3608360036013602360E36F8
:1013D0000450005E0550D8A0053C015E0650D8A020
:1013E000063C025E06340E120EA0FAEF09F00D80E4
:1013F00005EF0AF0045000260550D8B0053C012640
:101400000650D8B0062802260D900B2EE1EF09F009
:101410002BEF0AF0D8900036013602360E36045013
:10142000005E0550D8A0053C015E0650D8A0063CE1
:10143000025E06340E10010B0D26D8B00C2AD8B46B
:10144000082AD8A42BEF0AF008320C320D32032AF6
:10145000D8B43FEF0AF00AAE089E0850026E0C5056
:10146000016E0D50006E47EF0AF0010E70EC04F0B3
:1014700047EF0AF0020E11EC01F047EF0AF0040EFC
:101480005DEC03F047EF0AF0080EDBEC00F0120011
:101490000301566B55DC43DD890E046E410E056E6B
:1014A0001C0E066E810E076EF5DDCFDC12000250B9
:1014B00006180E6E086A096A0B6A035007644AEF41
:1014C0000BF006500A6E068E028E03500B6E07500C
:1014D000036E000E0B649AEF0AF00B50075ED8B44F
:1014E0003BEF0BF0070E076409EF0BF0075E00C03F
:1014F00008F001C000F002C001F0026A074E3BEFA5
:101500000BF00764DEEF0AF0075E00C008F001C0D0
:1015100000F0016A074E3BEF0BF00764BCEF0AF0E6
:10152000075E00C008F0006A074E3BEF0BF007644F
:10153000A3EF0AF00AC002F005C001F004C000F0F9
:10154000086A67EF0CF0030E0764AEEF0AF0075E5F
:1015500008380F0B086E074E3BEF0BF0D89008329F
:10156000074E3BEF0BF0D8900832074E3BEF0BF0E5
:10157000D89008323BEF0BF0030E0764CDEF0AF072
:10158000075E08380F0B086E0038F00B082600388D
:101590000F0B006E074E3BEF0BF0D8900032083275
:1015A000074E3BEF0BF0D89000320832074E3BEF6E
:1015B0000BF0D890003208323BEF0BF0030E0764BB
:1015C000F5EF0AF0075E08380F0B086E0038F00BD5
:1015D000082600380F0B006E0138F00B002601388A
:1015E0000F0B016E074E3BEF0BF0D890013200322B
:1015F0000832074E3BEF0BF0D89001320032083230
:10160000074E3BEF0BF0D8900132003208323BEF2F
:101610000BF0030E076426EF0BF0075E08380F0B84
:10162000086E0038F00B082600380F0B006E0138EA
:10163000F00B002601380F0B016E0238F00B01266B
:1016400002380F0B026E074E3BEF0BF0D8900232C0
:10165000013200320832074E3BEF0BF0D8900232D5
:10166000013200320832074E3BEF0BF0D8900232C5
:10167000013200320832096A000E0EAE2FEF0CF074
:10168000081E001E011E021E082A0022012202223C
:101690002FEF0CF00750D8A450EF0BF067EF0CF0D1
:1016A000096A02C00AF0028E068E0750035C076EBC
:1016B000D8B422EF0CF0070E0764F0EF0BF0075ED2
:1016C0000450096E0550046E0650056E066A074EFA
:1016D00022EF0CF0070E0764C5EF0BF0075E045015
:1016E000096E0550046E056A074E22EF0CF0070ED6
:1016F0000764A3EF0BF0075E0450096E046A074EFF
:1017000022EF0CF0070E07648AEF0BF00AC002F01C
:1017100067EF0CF0030E076495EF0BF0075E0938D6
:101720000F0B096E074E22EF0CF0D8900932074ECE
:1017300022EF0CF0D8900932074E22EF0CF0D8902F
:10174000093222EF0CF0030E0764B4EF0BF0075ED2
:1017500009380F0B096E0438F00B092604380F0BFB
:10176000046E074E22EF0CF0D89004320932074E77
:1017700022EF0CF0D89004320932074E22EF0CF021
:10178000D8900432093222EF0CF0030E0764DCEF2C
:101790000BF0075E09380F0B096E0438F00B0926B1
:1017A00004380F0B046E0538F00B042605380F0BB8
:1017B000056E074E22EF0CF0D89005320432093244
:1017C000074E22EF0CF0D890053204320932074E52
:1017D00022EF0CF0D89005320432093222EF0CF0DF
:1017E000030E07640DEF0CF0075E09380F0B096E4E
:1017F0000438F00B092604380F0B046E0538F00B83
:10180000042605380F0B056E0638F00B0526063842
:101810000F0B066E074E22EF0CF0D8900632053201
:1018200004320932074E22EF0CF0D890063205320E
:1018300004320932074E22EF0CF0D89006320532FE
:1018400004320932086A000E0EAE2FEF0CF0091EAA
:10185000041E051E061E092A04220522062209501E
:1018600008260450002205500122065002220EBE16
:1018700046EF0CF0D8A055EF0CF0023201320032E6
:101880000832033E55EF0CF061EF0CF0D8B05BEF7F
:101890000CF0000E081E001E011E021E082A002267
:1018A000012202220A7E5BEF0CF0010E0C6E74EC3A
:1018B00004F069EF0CF0020E0C6E74EC04F069EFAA
:1018C0000CF0040E0C6E5DEC03F069EF0CF0000EF2
:1018D0000C6E1200A6A202D00000FCD7A69C54C336
:1018E000A9FF55C3A8FFA69EA684F2CF00F0F29EE2
:1018F000550EA76EAA0EA76EA68200BE02D0F29E5B
:1019000001D0F28EA694A1B802D00000FCD7A19815
:101910001200040002017A51C819000ED8A4010E69
:10192000016EC751C619000ED8A4010E006E0150F9
:101930000012D8B403D17AC2C8F20301196B1A6B32
:1019400002017AA105D003011751192718511A2352
:1019500002017AA305D003011D5119271E511A2334
:1019600002017AA505D003011B5119271C511A2326
:1019700002017AA705D003011F51192720511A230C
:1019800002017AA905D003012751192728511A23EA
:1019900002017AAB05D003012551192726511A23DC
:1019A00002017AAD05D00301295119272A511A23C2
:1019B000030119C356F31AC357F30B0E586F030EE6
:1019C000596FB7EC06F00D51200A03E00DC3FEF28B
:1019D00003D0300E0201FE6F02012E0EFF6F0301D5
:1019E0000E51200A03E00EC300F302D0300E006F48
:1019F0000F51200A03E00FC301F302D0300E016F34
:101A00001251040A010ED8A4000E016E1251050AEB
:101A1000010ED8A4000E006E015000122AE002014F
:101A2000C751010A04E1040E0301546F03D00301FE
:101A3000060E546F0201C751C6190DE054C356F388
:101A4000100E0301576FDB0E586F020E596F080E10
:101A50005A6FCFEC07F054C356F3280E0301576FAB
:101A6000FE0E586F020E596F040E5A6FCFEC07F03E
:101A700065D003011251020A010ED8A4000E016EB6
:101A80001251030A010ED8A4000E006E015000127C
:101A900029E00201C751010A03E10301546B03D09D
:101AA0000301010E546F0201C751C6190DE054C362
:101AB00056F3090E0301576FD20E586F020E596F7D
:101AC000080E5A6FCFEC07F054C356F30B0E030108
:101AD000576FFE0E586F020E596F040E5A6FCFECFF
:101AE00007F02CD003011251000A28E00201C7516F
:101AF000010A03E10301546B03D00301010E546F8B
:101B00000201C751C6190DE054C356F3090E030173
:101B1000576FCA0E586F020E596F070E5A6FCFECEF
:101B200007F054C356F30B0E0301576FFE0E586FA8
:101B3000020E596F040E5A6FCFEC07F0020190515C
:101B4000C919000ED8A4010E016EC751C619000EA6
:101B5000D8A4010E006E01500012D8B4F8D090C283
:101B6000C9F20301196B1A6B020190A105D00301A0
:101B70002351192724511A23020190A305D00301F0
:101B80002151192722511A23020190A507D0EC51A7
:101B9000030119270201ED5103011A23020190A745
:101BA00007D0EA51030119270201EB5103011A235F
:101BB000020190A907D0E851030119270201E95158
:101BC00003011A23020190AB07D0F051030119273A
:101BD0000201F15103011A23020190AD07D0EE5129
:101BE000030119270201EF5103011A23030119C34D
:101BF00056F31AC357F30B0E586F030E596FB7EC19
:101C000006F00DC3FEF20EC3FFF20FC300F310C3C4
:101C100001F31251040A010ED8A4000E016E1251F4
:101C2000050A010ED8A4000E006E015000122AE031
:101C30000201C751010A04E1060E0301546F03D0EB
:101C40000301040E546F0201C751C6190DE054C3BD
:101C500056F3100E0301576FD50E586F000E596FD3
:101C6000080E5A6FCFEC07F054C356F3280E030149
:101C7000576FFE0E586F020E596F040E5A6FCFEC5D
:101C800007F065D003011251020A010ED8A4000E1C
:101C9000016E1251030A010ED8A4000E006E01500D
:101CA000001229E00201C751010A04E1010E0301FB
:101CB000546F02D00301546B0201C751C6190DE0E5
:101CC00054C356F3090E0301576FCC0E586F000E24
:101CD000596F080E5A6FCFEC07F054C356F30B0E32
:101CE0000301576FFE0E586F020E596F040E5A6FA4
:101CF000CFEC07F02CD003011251000A28E00201BA
:101D0000C751010A04E1010E0301546F02D003011F
:101D1000546B0201C751C6190DE054C356F3090EA6
:101D20000301576FBE0E586F000E596F070E5A6FA2
:101D3000CFEC07F054C356F30B0E0301576FFE0EA2
:101D4000586F020E596F040E5A6FCFEC07F0040063
:101D5000C7C2C6F20201C051000AD8A489D003014B
:101D60001251040A010ED8A4000E016E1251050A88
:101D7000010ED8A4000E006E015000123BE00001DD
:101D8000BD53010ED8A4000E006E0201C35100160F
:101D90000DE00301566B700E576FBB0E586F000EAF
:101DA000596F010E5A6FCFEC07F023D00201C353D5
:101DB000010ED8A4000E006E0001BD5100160DE00A
:101DC0000301566B700E576FCA0E586F000E596F95
:101DD000010E5A6FCFEC07F00CD00301566B700E5A
:101DE000576FC80E586F000E596F010E5A6FCFEC27
:101DF00007F03ED003011251000A3AE00001BD5342
:101E0000010ED8A4000E006E0201C35100160DE0B1
:101E10000301566B080E576FC60E586F000E596FB0
:101E2000010E5A6FCFEC07F023D00201C353010E0D
:101E3000D8A4000E006E0001BD5100160DE0030194
:101E4000566B080E576FF20E586F000E596F010E49
:101E50005A6FCFEC07F00CD00301566B080E576F8A
:101E6000F00E586F000E596F010E5A6FCFEC07F04D
:101E700004001200030E0C6E950E0D6E0D2EFED793
:101E80000C2EFCD71200010E0301566FA0EC06F0D9
:101E90008FEC07F0890E046E410E056E1C0E066E67
:101EA000810E076E4AEC08F025EC07F0120054C3CF
:101EB00000F055C301F0030E046E000E056EF5EC44
:101EC00003F000C054F301C055F3800E026E800E83
:101ED0000118025C02E10050500803E3006A016A45
:101EE000BCD0800E006E800E03015519005C02E12B
:101EF0005451AB0805E3F40E5427000E5523A9D026
:101F0000800E010A006E800E5519005C02E15451EA
:101F1000480805E3FE0E5427000E55239AD0800E84
:101F2000020A006E800E5519005C02E15451460809
:101F300005E3180E5427010E55238BD0800E030A9B
:101F4000006E800E5519005C02E15451340805E31F
:101F5000290E5427010E55237CD0800E040A006EF2
:101F6000800E5519005C02E154514C0805E3360E11
:101F70005427010E55236DD0800E080A006E800E86
:101F80005519005C02E15451850805E3AE0E542753
:101F9000010E55235ED0800E0C0A006E800E55197E
:101FA000005C02E15451FA0805E3E40E5427010EE7
:101FB00055234FD0800E120A006E800E5519005C1A
:101FC00002E154510F0805E3120E5427020E552367
:101FD00040D0800E160A006E800E5519005C02E19A
:101FE0005451E60805E3880E5427020E552331D0DC
:101FF000800E1B0A006E800E5519005C02E15451E0
:10200000EA0805E3E70E5427020E552322D0800E7E
:10201000210A006E800E5519005C02E15451360809
:1020200005E3200E5427030E552313D0800E290AF2
:10203000006E800E5519005C02E15451040805E35E
:10204000340E5427030E552304D0520E5427030E8A
:10205000552354C300F055C301F0120000C008F02E
:102060000150006E016A026A036A0B6A0C6A016A17
:10207000026A036A960E036E0A6A00AE46EF10F01B
:10208000081E001E082AD8B4002A0A8E00C001F0DB
:1020900008C000F0086A026A69EC03F01200005000
:1020A000086E0150006E0250016E0350026E036A0A
:1020B0000B6A0C6A9E0E036E0A6A02AE6CEF10F099
:1020C000081E001E011E021E082AD8B4002AD8B419
:1020D000012AD8B4022A0A8E020E0C6E74EC04F0A7
:1020E000120002017A6B906B0301566B1DEC04F039
:1020F00090C256F3A4EC07F005C360F306C361F386
:1021000018EC01F01200040048EC0AF000C048F39B
:1021100001C049F3000E01BEFF0E03014A6F4B6F71
:10212000B2DE00C04CF301C04DF3000E01BEFF0E45
:1021300003014E6F4F6F02017B51010A0FE148C34B
:1021400054F349C355F3B3DE89DF00C050F301C037
:1021500051F302C052F303C053F311D048C300F04F
:1021600049C301F04AC302F04BC303F098DF00C03B
:1021700050F301C051F302C052F303C053F3800E79
:1021800003014F19006E800E4B19005C08E14A51A3
:102190004E5D05E149514D5D02E148514C5D08E35A
:1021A000E70E486F030E496F000E4A6F4B6F45D024
:1021B0004C514825006E4D514921016E4E514A2126
:1021C000026E4F514B21036E640E046E000E056EBD
:1021D000066E076EE8EC00F048C304F049C305F052
:1021E0004AC306F04BC307F04C51045E4D51055AEB
:1021F0004E51065A4F51075ADDEC08F000C048F323
:1022000001C049F302C04AF303C04BF3800E046ED1
:10221000800E0318045C08E10250000805E101503B
:10222000030802E10050E70808E2E70E0301486FE7
:10223000030E496F000E4A6F4B6F50C300F051C33D
:1022400001F052C302F053C303F0000E046E000EFF
:10225000056E200E066E820E076E4AEC08F0000E28
:10226000046E000E056E7A0E066E880E076E8AECFE
:1022700009F000C050F301C051F302C052F303C093
:1022800053F3F40E046EFD0E056E340E066E7F0ED3
:10229000076E8AEC09F000C050F301C051F302C090
:1022A00052F303C053F300C004F001C005F002C0B4
:1022B00006F003C007F04AEC08F0000E046E000EB2
:1022C000056E200E066E810E076E8AEC09F000C0C6
:1022D00050F301C051F302C052F303C053F3000E98
:1022E000046E000E056E000E066E7E0E076E57EC35
:1022F0000AF000C050F301C051F302C052F303C012
:1023000053F325EC07F000C007F301C008F3800E7B
:102310000118026E800E025C02E10A0E005C06E209
:10232000010E0301136F000E146F19D00301800E0C
:102330004B19006E800E005C08E1000E4A5D05E15D
:10234000000E495D02E1640E485D05E2E70E136F81
:10235000030E146F04D048C313F349C314F31200DF
:102360000134083609360450085E0550D8A0053CF3
:10237000095E003601360F0E0C6E01340836093640
:10238000045000A006D0085E0550D8A0053C095EA8
:1023900005D008260550D8B0053C09260036013680
:1023A0000C2EEBD700B006D0045008260550D8B04C
:1023B000053C09260000120094DEFF0E546F556B99
:1023C0006AEC0CF0FE0E0301546F556B6AEC0CF0D6
:1023D000FD0E0301546F556B6AEC0CF089EC0CF0A8
:1023E00003011251000A02E18A8C8A8E899E898C2F
:1023F000136B146B076B086B0201BE6BBF6B0301A1
:102400001251040A010ED8A4000E016E1251050AE1
:10241000010ED8A4000E006E0150001236E0020E2C
:10242000566F100E576FE70E586F000E596F080E5B
:102430005A6FCFEC07F004000D0E0B6E2D0E0C6ED4
:10244000D70E0D6E0D2EFED70C2EFCD70B2EFAD705
:1024500000000000020E0301566F100E576FDE0ED3
:10246000586F000E596F080E5A6FCFEC07F003013A
:10247000566B100E576FB20E586F000E596F080E44
:102480005A6FCFEC07F0040036D003011251000A56
:1024900032E0010E566F576B500E586F000E596F99
:1024A000080E5A6FCFEC07F004000D0E0B6E2D0EC8
:1024B0000C6ED70E0D6E0D2EFED70C2EFCD70B2EEC
:1024C000FAD700000000010E0301566F576B470E4C
:1024D000586F000E596F080E5A6FCFEC07F00301CA
:1024E000566B576B3E0E586F000E596F080E5A6FA1
:1024F000CFEC07F00400120003014E6B4AC301F059
:10250000010E006E015004E000360090FF0FFBD773
:1025100000C04DF348C3E9FF49C3EAFF0050EE1481
:10252000016E0152010ED8A4000E006E4C51001A2B
:1025300018E04B51000804E29DDC9CDC4B07F9D706
:1025400048C3E9FF49C3EAFF4D51EE14016E015241
:10255000010ED8A4000E006E4C51001A02E0FF0ECE
:102560004E6F4EC300F01200CEDD800E0819026ED1
:10257000800E1619025C02E11551075D010ED8B0FC
:10258000000E026E800E2C19016E800E0819015C7F
:1025900002E107512B5D010ED8B0000E016E800ED6
:1025A000006E800E2C19005C02E12B510008010E18
:1025B000D8B0000E006E01500016025000122BE041
:1025C0000400A1DD810E486F0F0E496F4A6B050EA6
:1025D0004B6F010E4C6F90DF005203E0010E0201C1
:1025E000E56F0201E551010A010ED8A4000E0301B6
:1025F000476F810E486F0F0E496F4A6B050E4B6F88
:102600004C6B7ADF4751001605E0D6DE0301136BF1
:10261000146B01D0AAD712000450000A08E105503B
:10262000000A05E1FF0E006E7F0E016E57D00D6AA5
:10263000096A086A01500010D8B4000C015005184E
:102640000A6E0ABE0D1E0B6A05AE05D0041E051EDD
:10265000042AD8B4052A01AE05D0001E011E002AA6
:10266000D8B4012A015005100A6E0ABE10D078DED7
:102670000BB020D00DAE000C001E011E002AD8B4F5
:10268000012A081E091E082AD8B4092A000C05AE22
:102690000DD001BE07D00150096E0050086E016ACE
:1026A000006AE8D7016A006A002A000C011E001EB9
:1026B0000B2ADDD7082AD8B4092A0450085CD8A40C
:1026C000D9D70550095CD8A4D5D7096A086A002A69
:1026D000D8B4012A01AECED70000FF0C1200030EC1
:1026E0000301466F0201906B0301566BA4EC07F0E7
:1026F00046C392F239DF000E141902E1000E1319DD
:1027000001E186D0140E046E000E056E13C300F0B6
:1027100014C301F081DF005003011325446F015001
:102720001421456F46C343F343511F08D8A06CD012
:10273000435102019103F3CF56F3A4EC07F014DFE9
:10274000000E141902E1000E131901E161D0800E90
:102750001419006E800E4519005C02E14451135DAE
:1027600051E2140E046E000E056E13C300F014C384
:1027700001F052DF005003011325446F0150142172
:10278000456F435102019103F3CF90F246C392F299
:10279000800E03011419006E800E005C02E1780EB9
:1027A000135D01E231D046514325026E02C043F36E
:1027B00002017D51000A010ED8A4000E016E0250E4
:1027C000090A010ED8A4000E006E0150001604E0A4
:1027D000080E0301436F15D002017D51000A010E5E
:1027E000D8A4000E016E03014351110A010ED8A4B2
:1027F000000E006E0150001604E0100E436F040E30
:10280000466F01D001D090D790C256F3A4EC07F0E8
:102810001200020192519103F3CF00F000C03DF38A
:1028200000509025046E04C03FF3050E026E91C265
:1028300000F0000E016E025005E0003600900136F7
:10284000FF0FFAD7010E005C026E000E0158036EF6
:10285000800E0318006E800E005C02E10450025CE2
:102860000DE2050E006E91C23FF3005005E003013A
:102870003F373F91FF0FFAD703013F070201905105
:1028800003013D5D06E23D510201905D0301406F91
:1028900001D0406B40C390F240C356F3A4EC07F064
:1028A00063DE000E141902E1000E131901E167D076
:1028B00013C341F314C342F30201915103014025B4
:1028C0003E6F3E513F5D57E33EC356F3A4EC07F025
:1028D0004BDE000E141902E1000E131901E14FD076
:1028E000800E1419006E800E4219005C02E1415105
:1028F000135D0BE3340E0C6EF10E0D6E0D2EFED734
:102900000C2EFCD7000000002FDE800E1419006E84
:10291000800E4219005C02E14151135D0BE3340E5D
:102920000C6EF10E0D6E0D2EFED70C2EFCD7000096
:1029300000001ADE800E1419006E800E4219005C31
:1029400002E14151135D11E213C341F314C342F399
:102950003EC390F2800E1419006E800E005C02E1FE
:10296000780E135D01E207D001D005D0020191512C
:1029700003013E27A6D790C256F3A4EC07F012003D
:1029800003013DB102D08B9001D08B8005C360F371
:1029900006C361F318EC01F01200030E0301426F4D
:1029A0003E6B42C379F2030E3F6F140E046E000EAD
:1029B000056E13C300F014C301F02EDE00500301B6
:1029C0001325406F01501421416F42C33DF33D5127
:1029D0001F08D8A071D03D5102017803F3CF56F300
:1029E0001DEC04F07CDEC0DD000E141902E1000EC7
:1029F000131901E177D0800E1419006E800E411971
:102A0000005C02E14051135D55E2140E046E000EAD
:102A1000056E13C300F014C301F0FEDD0050030186
:102A20001325406F01501421416F3D51020178037D
:102A3000F3CF7AF290C23EF342C379F292C23FF3EF
:102A4000800E03011419006E800E005C02E1780E06
:102A5000135D01E231D042513D25026E02C03DF3CB
:102A600002017C51000A010ED8A4000E016E025032
:102A7000090A010ED8A4000E006E0150001604E0F1
:102A8000080E03013D6F15D002017C51000A010EB2
:102A9000D8A4000E016E03013D51110A010ED8A405
:102AA000000E006E0150001604E0100E3D6F040E83
:102AB000426F01D001D08BD73EC390F27AC256F359
:102AC0001DEC04F090C256F3A4EC07F03FC392F261
:102AD000340E0C6EF10E0D6E0D2EFED70C2EFCD7A3
:102AE000000000001200020179517803F3CF00F0DA
:102AF00000C03DF300507A25046E04C03FF3050E7C
:102B0000026E78C200F0000E016E025005E0003641
:102B100000900136FF0FFAD7010E005C026E000E26
:102B20000158036E800E0318006E800E005C02E1F7
:102B30000450025C0DE2050E006E78C23FF30050B7
:102B400005E003013F373F91FF0FFAD703013F072D
:102B500002017A5103013D5D06E23D5102017A5DB9
:102B60000301406F01D0406B40C37AF240C356F37B
:102B70001DEC04F0F9DC000E141902E1000E13192B
:102B800001E167D013C341F314C342F3020178514A
:102B9000030140253E6F3E513F5D57E33EC356F370
:102BA0001DEC04F0E1DC000E141902E1000E131913
:102BB00001E14FD0800E1419006E800E4219005CA6
:102BC00002E14151135D0BE3340E0C6EF10E0D6EFC
:102BD0000D2EFED70C2EFCD700000000C5DC800EA9
:102BE0001419006E800E4219005C02E14151135D20
:102BF0000BE3340E0C6EF10E0D6E0D2EFED70C2E67
:102C0000FCD700000000B0DC800E1419006E800EAE
:102C10004219005C02E14151135D11E213C341F31B
:102C200014C342F33EC37AF2800E1419006E800E74
:102C3000005C02E1780E135D01E207D001D005D0FF
:102C40000201785103013E27A6D77AC256F31DEC44
:102C500004F01200810E0301486F0F0E496F4A6B9A
:102C6000320E4B6F4C6B48DC00C037F3810E486F5F
:102C70000F0E496F010E4A6F320E4B6F4C6B3CDCEE
:102C800000503713810E486F0F0E496F020E4A6FC6
:102C9000320E4B6F4C6B30DC3751001203E0010EEB
:102CA0000201956F120013C337F314C338F375DEB6
:102CB000000E141902E1000E131903E171EC10F07B
:102CC00001D152DC800E1419006E800E005C02E10E
:102CD000780E135D01E2F6D006DF000E141902E152
:102CE000000E131903E171EC10F0ECD03DDC800E06
:102CF0001419006E800E005C02E1780E135D01E293
:102D0000E1D087DD000E141902E1000E131903E172
:102D100071EC10F0D7D028DC800E1419006E800EF4
:102D2000005C02E1780E135D01E2CCD0800E141934
:102D3000016E800E015C02E1C80E135D010ED8B079
:102D4000000E016E800E1419006E800E3819005CA2
:102D500002E13751135D010ED8B0000E006E005035
:102D60000114036E1351375D016E14513859026E10
:102D7000800E006E800E0218005C02E101506408B3
:102D8000010ED8B0000E006E0350001601E09AD07C
:102D900013C337F314C338F37AC239F3000E3A6F12
:102DA00090C23BF3000E3C6F0201C751010A02E1E1
:102DB000C76B02D0010EC76F71EC10F0C7C23DF3B4
:102DC000DFDD020E0B6E040E0C6EBA0E0D6E0D2EB4
:102DD000FED70C2EFCD70B2EFAD70000B4EC12F065
:102DE000800E1419006E800E005C02E1780E135DF7
:102DF00001E268D0D2DD000E141902E1000E1319B1
:102E000003E171EC10F05ED0B4EC12F0800E1419F6
:102E1000006E800E005C02E1780E135D01E252D07C
:102E200062DE000E141902E1000E131903E171ECC9
:102E300010F048D0B4EC12F0800E1419006E800E21
:102E4000005C02E1780E135D01E23CD0E2DC000E92
:102E5000141902E1000E131903E171EC10F032D0E5
:102E6000B4EC12F0800E1419006E800E005C02E1CA
:102E7000780E135D01E226D0800E3819006E800EA8
:102E80001419005C02E11351375D1BE20201C751C6
:102E9000010A02E1C76B02D0010EC76FC7C23DF342
:102EA0006FDD39C37AF23BC390F239C356F31DECA0
:102EB00004F090C256F3A4EC07F037C313F338C301
:102EC00014F30400120004000301385102019419A4
:102ED00003E1935103013719D8B480D0030137C3FC
:102EE00093F238C394F2000E381902E1010E37193B
:102EF00030E11251040A010ED8A4000E016E1251E5
:102F0000050A010ED8A4000E006E015000120DE05B
:102F1000020E566F400E576F9B0E586F020E596F80
:102F2000040E5A6FCFEC07F010D003011251000AC3
:102F30000CE0010E566F040E576F960E586F020E7E
:102F4000596F040E5A6FCFEC07F00201936B946B2C
:102F500045D037C393F238C394F237C356F338C31E
:102F600057F30B0E0301586F030E596FB7EC06F0C1
:102F70000EC3FEF22E0E0201FF6F0FC300F310C34B
:102F800001F303011251040A010ED8A4000E016ED0
:102F90001251050A010ED8A4000E006E0150001255
:102FA0000DE0020E566F400E576FFE0E586F020E68
:102FB000596F040E5A6FCFEC07F010D00301125175
:102FC000000A0CE0010E566F040E576FFE0E586F8C
:102FD000020E596F040E5A6FCFEC07F00400120076
:102FE000040000019351050A04E1010E0201786F0B
:102FF0000FD000019351060A04E1020E0201786F1E
:1030000007D000019351070A03E1040E0201786F13
:1030100000019251050A04E1010E0201916F0FD0E7
:1030200000019251060A04E1020E0201916F07D0DD
:1030300000019251070A03E1040E0201916F02019F
:10304000E56BB4EC12F0800E1419006E800E005C7B
:1030500002E16E0E135D01E275D071EC10F0020E0C
:103060000B6E040E0C6EBA0E0D6E0D2EFED70C2ECE
:10307000FCD70B2EFAD70000B4EC12F0800E141916
:10308000006E800E005C02E16E0E135D01E25AD00C
:10309000800E016E800E0201E719015C02E1E6512B
:1030A0006E08010ED8B0000E016E800EE719006E9A
:1030B000800E03011419005C03E113510201E65D67
:1030C000010ED8B0000E006E0150001601E03AD09B
:1030D000EADD000E141902E1000E131903E171EC90
:1030E00010F030D0800E1419006E800E005C02E1EA
:1030F000780E135D01E226D000019251050A010EFF
:10310000D8A4000E016E9351050A010ED8A4000E3A
:10311000006E0150001601E015D09351050806E23B
:1031200078C279F2010E0201786FDDDC0001925164
:10313000050807E291C292F2010E0201916F09ECBB
:1031400014F00400120045EC00F0F2C26FF30EEC34
:1031500000F0800E03016F6F0EEC00F031C36FF3CF
:103160000EEC00F0C4EC00F012000301356B366B7E
:10317000640E095D326F000E0A59336F076B086BDE
:10318000010E0201C16F000EC26F0400C051010A9E
:1031900004E1280E0301346F03D00301780E346F6D
:1031A000316B3451315D4EE20201C051000A010E13
:1031B000D8A4000E016E81B002D0068001D0069026
:1031C00081B202D0D88001D0D89006B003D002E2FC
:1031D000069001D0068081B402D0D88001D0D8906A
:1031E00006B003D002E2069001D00680006A06B065
:1031F000002A0150001607E02DDD02019551010A59
:1032000002E1956B38D383EC10F0800E3619006E16
:10321000800E0819005C02E10751355D08E207C322
:1032200035F308C336F313C3C1F214C3C2F2100E50
:103230000C6E940E0D6E0D2EFED70C2EFCD70000DA
:10324000312BAFD7040035C3C4F236C3C5F2C1C2B7
:1032500037F3C2C238F337DE800E0201C219006EA6
:10326000800E03010A19005C03E109510201C15DEE
:103270000201000ED8B0010E006E0050C315056E9D
:10328000800EBF19036E800EC219035C02E1C151AA
:10329000BE5D010ED8B0000E036EBE51C15D016E61
:1032A000BF51C259026E800E03013319006E800EA9
:1032B0000218005C02E10150325D010ED8B0000E30
:1032C000006E00500314046E800E0201C219036EDA
:1032D000800EBF19035C02E1BE51C15D010ED8B082
:1032E000000E036EC151BE5D016EC251BF59026E28
:1032F000800E03013319006E800E0218005C02E19B
:103300000150325D010ED8B0000E006E0350001661
:1033100000500410016E0201BF51030A02E1E70EE2
:10332000BE19010ED8A4000E006E01500012055007
:10333000001602E0010EA26FC051000A010ED8A4CF
:10334000000E016E81B002D0068001D0069081B2DD
:1033500002D0D88001D0D89006B003D002E2069007
:1033600001D0068081B402D0D88001D0D89006B0B8
:1033700003D002E2069001D00680006A06B0002A5F
:103380000150001607E066DC02019551010A02E1D6
:10339000956B71D20201C551A11902E1A051C41966
:1033A000D8B477D0C4C2A0F2C5C2A1F2800EC519AC
:1033B000006E800E005C02E1640EC45D1EE3050E2B
:1033C000C425006E000EC521016E00C0C4F201C00C
:1033D000C5F200C056F301C057F30B0E0301586F3E
:1033E000030E596FB7EC06F00DC3FEF20EC3FFF2E9
:1033F0000FC300F3570E016F22D00301C4C256F36E
:10340000C5C257F30B0E586F030E596FB7EC06F099
:103410000F51200A03E00FC3FEF203D0300E020169
:10342000FE6F02012E0EFF6F03011051200A03E010
:1034300010C300F302D0300E006F570E016F12510F
:10344000040A010ED8A4000E016E1251050A010EE5
:10345000D8A4000E006E015000120CE0566B400E16
:10346000576FFE0E586F020E596F040E5A6FCFEC55
:1034700007F00FD003011251000A0BE0566B040E47
:10348000576FFE0E586F020E596F040E5A6FCFEC35
:1034900007F00201C051000A010ED8A4000E016E0F
:1034A00081B002D0068001D0069081B202D0D880CF
:1034B00001D0D89006B003D002E2069001D0068079
:1034C00081B402D0D88001D0D89006B003D002E2F7
:1034D000069001D00680006A06B0002A015000164E
:1034E00008E02AEC16F002019551010A02E1956B01
:1034F000C2D102010400800E050A006E800EC519BB
:10350000005C02E1C451DC08D8B0B5D1030112510E
:10351000040A010ED8A4000E016E1251050A010E14
:10352000D8A4000E006E01500012D8B4C7D0020E0D
:10353000566F100E576FA30E586F020E596F080E7C
:103540005A6FCFEC07F0030E0B6E080E0C6E770E61
:103550000D6E0D2EFED70C2EFCD70B2EFAD7020EB9
:103560000301566F100E576FB50E586F020E596F4C
:10357000080E5A6FCFEC07F00B0E0B6E260E0C6E7A
:103580005D0E0D6E0D2EFED70C2EFCD70B2EFAD72E
:10359000000000000400020E0301566F100E576F6A
:1035A000AC0E586F020E596F080E5A6FCFEC07F031
:1035B000070E0B6E170E0C6E6A0E0D6E0D2EFED7DB
:1035C0000C2EFCD70B2EFAD70000020E0301566F0B
:1035D000100E576F540E586F020E596F080E5A6F27
:1035E000CFEC07F00B0E0B6E260E0C6E5D0E0D6E03
:1035F0000D2EFED70C2EFCD70B2EFAD700000000A4
:103600000400020E0301566F100E576F4B0E586FD9
:10361000020E596F080E5A6FCFEC07F0070E0B6EB3
:10362000170E0C6E6A0E0D6E0D2EFED70C2EFCD7EB
:103630000B2EFAD70000020E0301566F100E576FC3
:103640005D0E586F020E596F080E5A6FCFEC07F0DF
:103650000B0E0B6E260E0C6E5D0E0D6E0D2EFED734
:103660000C2EFCD70B2EFAD7000000000400020E2F
:103670000301566F100E576F6F0E586F020E596F81
:10368000080E5A6FCFEC07F0030E0B6E080E0C6E8F
:10369000770E0D6E0D2EFED70C2EFCD70B2EFAD703
:1036A000020E0301566F100E576F660E586F020E12
:1036B000596F080E5A6FCFEC07F0C3D003011251B7
:1036C000000AD8B4BED0010E566F576B420E586F29
:1036D000020E596F080E5A6FCFEC07F0030E0B6EF7
:1036E000080E0C6E770E0D6E0D2EFED70C2EFCD72D
:1036F0000B2EFAD7010E0301566F576B1E0E586F33
:10370000020E596F080E5A6FCFEC07F00B0E0B6EBE
:10371000260E0C6E5D0E0D6E0D2EFED70C2EFCD7F8
:103720000B2EFAD7000000000400010E0301566FB3
:10373000576B150E586F020E596F080E5A6FCFEC6B
:1037400007F0070E0B6E170E0C6E6A0E0D6E0D2E27
:10375000FED70C2EFCD70B2EFAD70000010E03016A
:10376000566F576B270E586F020E596F080E5A6F1F
:10377000CFEC07F00B0E0B6E260E0C6E5D0E0D6E71
:103780000D2EFED70C2EFCD70B2EFAD70000000012
:103790000400010E0301566F576B390E586F020E6D
:1037A000596F080E5A6FCFEC07F0070E0B6E170E0D
:1037B0000C6E6A0E0D6E0D2EFED70C2EFCD70B2E46
:1037C000FAD70000010E0301566F576B300E586F89
:1037D000020E596F080E5A6FCFEC07F00B0E0B6EEE
:1037E000260E0C6E5D0E0D6E0D2EFED70C2EFCD728
:1037F0000B2EFAD7000000000400010E0301566FE3
:10380000576B870E586F020E596F080E5A6FCFEC28
:1038100007F0030E0B6E080E0C6E770E0D6E0D2E5C
:10382000FED70C2EFCD70B2EFAD7010E0301566FD4
:10383000576B7E0E586F020E596F080E5A6FCFEC01
:1038400007F00B0E0B6E260E0C6E5D0E0D6E0D2E20
:10385000FED70C2EFCD70B2EFAD700000000040078
:10386000100E0201936F270E946FC1C237F3C2C2CC
:1038700038F363EC17F01200400E0201F56F0D0EE5
:10388000F66F560EF76F030EF86FC26A01013B1D0B
:10389000006E0050C116070EC012C08EC28012000A
:1038A00045EC00F0F2C26FF30EEC00F003016F6B19
:1038B0000EEC00F0AE0E03016F6F0EEC00F0020193
:1038C000FA51020A010ED8A4000E016EFA51030A41
:1038D000010ED8A4000E006E01500012D8B497D08B
:1038E000D50E03016F6F0EEC00F0800E03016F6FB9
:1038F0000EEC00F0A80E03016F6F0EEC00F03F0E0F
:1039000003016F6F0EEC00F0D30E03016F6F0EEC2E
:1039100000F00201FA51020A05E1FBC26FF30EEC5E
:1039200000F007D00201FB511F0F03016F6F0EEC77
:1039300000F0400E03016F6F0EEC00F08D0E0301DE
:103940006F6F0EEC00F0140E03016F6F0EEC00F0C1
:10395000810E03016F6F0EEC00F0B40E03016F6F68
:103960000EEC00F0D90E03016F6F0EEC00F0220E8A
:1039700003016F6F0EEC00F0200E03016F6F0EEC71
:1039800000F0020E03016F6F0EEC00F0210E030138
:103990006F6F0EEC00F003016F6B0EEC00F07F0E0A
:1039A00003016F6F0EEC00F02E0E03016F6F0EEC33
:1039B00000F00201FA51020A0BE1A00E03016F6F41
:1039C0000EEC00F0C00E03016F6F0EEC00F00AD099
:1039D000A10E03016F6F0EEC00F0C80E03016F6FB4
:1039E0000EEC00F0DA0E03016F6F0EEC00F0020E29
:1039F00003016F6F0EEC00F0DB0E03016F6F0EEC36
:103A000000F0400E03016F6F0EEC00F08AD0D50E6F
:103A100003016F6F0EEC00F0800E03016F6F0EEC70
:103A200000F0A80E03016F6F0EEC00F03F0E0301D3
:103A30006F6F0EEC00F0D30E03016F6F0EEC00F011
:103A4000FBC26FF30EEC00F0400E03016F6F0EEC43
:103A500000F08D0E03016F6F0EEC00F0140E0301E9
:103A60006F6F0EEC00F0810E03016F6F0EEC00F033
:103A7000FF0E03016F6F0EEC00F0D90E03016F6FA4
:103A80000EEC00F0F10E03016F6F0EEC00F0200E53
:103A900003016F6F0EEC00F0020E03016F6F0EEC6E
:103AA00000F0210E03016F6F0EEC00F003016F6B4D
:103AB0000EEC00F07F0E03016F6F0EEC00F02E0E87
:103AC00003016F6F0EEC00F00201FA51040A0BE1E2
:103AD000A00E03016F6F0EEC00F0C00E03016F6FBC
:103AE0000EEC00F00AD0A10E03016F6F0EEC00F097
:103AF000C80E03016F6F0EEC00F0DA0E03016F6F5A
:103B00000EEC00F0120E03016F6F0EEC00F0DB0EF6
:103B100003016F6F0EEC00F0400E03016F6F0EECAF
:103B200000F0A40E03016F6F0EEC00F0A60E03016F
:103B30006F6F0EEC00F0C4EC00F0030E0B6E080E7D
:103B40000C6E770E0D6E0D2EFED70C2EFCD70B2EA5
:103B5000FAD745EC00F0F2C26FF30EEC00F0400E25
:103B600003016F6F0EEC00F00201FA51020A010E20
:103B7000D8A4000E016EFA51030A010ED8A4000E5B
:103B8000006E0150001219E00301306B3051030840
:103B900013E330C36AF36B6B81EC00F003012F6B0E
:103BA0000301800E2F5D05E22F2B6F6B0EEC00F0F2
:103BB000F7D70301302BEAD718D00301306B30510F
:103BC000070813E330C36AF36B6B81EC00F0030169
:103BD0002F6B0301800E2F5D05E22F2B6F6B0EEC18
:103BE00000F0F7D70301302BEAD7C4EC00F0AF0E9A
:103BF0000301316FA3EC18F012000400030112510D
:103C0000040A010ED8A4000E016E1251050A010E1D
:103C1000D8A4000E006E0150001248E0566B100E42
:103C2000576FDA0E586F010E596F080E5A6FCFECAE
:103C300007F0020E0301566F100E576FD10E586F2A
:103C4000010E596F080E5A6FCFEC07F0040E0301F6
:103C5000566F100E576FC80E586F010E596F080E31
:103C60005A6FCFEC07F0060E0301566F100E576F18
:103C70003C0E586F010E596F080E5A6FCFEC07F0CB
:103C80000201C053010ED8A4000E006EC3510016ED
:103C90000CE00301566B700E576F200E586F010E2B
:103CA000596F010E5A6FCFEC07F065D00301125126
:103CB000000A61E0566B576B170E586F010E596F73
:103CC000080E5A6FCFEC07F0010E0301566F576BC9
:103CD0000E0E586F010E596F080E5A6FCFEC07F099
:103CE00003011251010A19E1566B090E576F330E89
:103CF000586F010E596F070E5A6FCFEC07F0010E87
:103D00000301566F090E576F2B0E586F010E596F36
:103D1000070E5A6FCFEC07F019D00301566B090E4E
:103D2000576F220E586F010E596F080E5A6FCFEC65
:103D300007F0010E0301566F090E576F050E586FFD
:103D4000010E596F080E5A6FCFEC07F00201C053F5
:103D5000010ED8A4000E006EC35100160CE0030142
:103D6000566B080E576F010E586F010E596F010EFA
:103D70005A6FCFEC07F004000201C86BC96B89ECE5
:103D80000CF012002FC300F00032009E0032009EA3
:103D90000032009E0032009E0A0E0002F3CF01F0B6
:103DA0000F0E03012F15006E0150002612000400B3
:103DB00003011251000A02E18A8C8A8E1251040A10
:103DC000010ED8A4000E016E1251050A010ED8A4EE
:103DD000000E006E0150001219E0566B400E576F36
:103DE000E30E586F010E596F040E5A6FCFEC07F0B7
:103DF000020E0301566F400E576FC30E586F010E2F
:103E0000596F040E5A6FCFEC07F01CD0030112510A
:103E1000000A18E0566B040E576FBE0E586F010E65
:103E2000596F040E5A6FCFEC07F0010E0301566F65
:103E3000040E576FB90E586F010E596F040E5A6F6A
:103E4000CFEC07F0F0EC17F0FF0E0301546F90C2B7
:103E500055F36AEC0CF0FE0E0301546F7AC255F371
:103E60006AEC0CF0FD0E0301546FC7C255F36AEC07
:103E70000CF003011251000A18E1800E006E800E52
:103E80001419005C02E11351960802E38A9C0DD0DC
:103E9000800E006E800E1419005C02E11351FA08C6
:103EA00003E3819C819E01D0819E100E0201936FDD
:103EB000270E946F100EA06F270EA16FB5EC18F0AF
:103EC00013C3BEF214C3BFF289EC0CF0899E898C37
:103ED00004001200A69C2FC3A9FFA69EA680A8CF0F
:103EE00000F012000900F5CFE6FF0006FBE1010635
:103EF000F9E11200070EB46E600ED36E9B8C806ADF
:103F0000816A826A896A8A6A8B6A030E926E070ED8
:103F1000936E946AB1DC0D0EC16EF19EF29E12009A
:103F20000400010E03012F6FD5DF00C012F3020E53
:103F30002F6FD0DF0050010A03E1010E0201C36FB1
:103F4000030E03012F6FC6DF00C02FF31BDF00C07D
:103F500005F3000E066F040E2F6FBCDF00C02FF3B9
:103F600011DF0A0E0002F3CF09F3F4CF0AF3050EB6
:103F70002F6FB0DF00C02FF305DF0A0E0002F3CF72
:103F800015F3F4CF16F3060E2F6FA4DF00C02FF346
:103F9000F9DE0A0E0002F3CF2BF3F4CF2CF3090E57
:103FA0002F6F98DF00C02FF3EDDE0A0E0002F3CF73
:103FB000E6F2F4CFE7F20A0E2F6F8CDF00C093F029
:103FC0000B0E2F6F87DF00C07CF20C0E2F6F82DF8D
:103FD00000C092F00D0E2F6F7DDF00C07DF20E0E3F
:103FE0002F6F78DF00C07BF20F0E2F6F73DF00C0E2
:103FF000E4F20400100E2F6F6DDF00C02FF3C2DE5D
:10400000640E0002F3CF2DF3F4CF2EF3110E2F6FB9
:1040100061DF00C02FF3B6DE00502D25176F000EB4
:104020002E21186F120E2F6F55DF00C02FF3AADE5E
:10403000640E0002F3CF2DF3F4CF2EF3130E2F6F87
:1040400049DF00C02FF39EDE00502D251D6F000EAE
:104050002E211E6F140E2F6F3DDF00C02FF392DE56
:10406000640E0002F3CF2DF3F4CF2EF3150E2F6F55
:1040700031DF00C02FF386DE00502D251B6F000EB0
:104080002E211C6F160E2F6F25DF00C02FF37ADE56
:10409000640E0002F3CF2DF3F4CF2EF3170E2F6F23
:1040A00019DF00C02FF36EDE00502D251F6F000EAC
:1040B0002E21206F180E2F6F0DDF00C02FF362DE50
:1040C000640E0002F3CF2DF3F4CF2EF3190E2F6FF1
:1040D00001DF00C02FF356DE00502D25276F000EA4
:1040E0002E21286F1A0E2F6FF5DE00C02FF34ADE47
:1040F000640E0002F3CF2DF3F4CF2EF31B0E2F6FBF
:10410000E9DE00C02FF33EDE00502D25256F000EA6
:104110002E21266F1C0E2F6FDDDE00C02FF332DE46
:10412000640E0002F3CF2DF3F4CF2EF31D0E2F6F8C
:10413000D1DE00C02FF326DE00502D25296F000EA2
:104140002E212A6F200E2F6FC5DE00C02FF31ADE3E
:10415000640E0002F3CF2DF3F4CF2EF3210E2F6F58
:10416000B9DE00C02FF30EDE00502D25236F000EA8
:104170002E21246F220E2F6FADDE00C02FF302DE42
:10418000640E0002F3CF2DF3F4CF2EF3230E2F6F26
:10419000A1DE00C02FF3F6DD00502D25216F000EAB
:1041A0002E21226F240E2F6F95DE00C02FF3EADD43
:1041B000640E0002F3CF2DF3F4CF2EF3250E2F6FF4
:1041C00089DE00C02FF3DEDD00502D250201EC6FEB
:1041D000000E03012E210201ED6F260E03012F6F49
:1041E00079DE00C02FF3CEDD640E0002F3CF2DF395
:1041F000F4CF2EF3270E2F6F6DDE00C02FF3C2DD3C
:1042000000502D250201EA6F000E03012E2102014C
:10421000EB6F280E03012F6F5DDE00C02FF3B2DDC0
:10422000640E0002F3CF2DF3F4CF2EF3290E2F6F7F
:1042300051DE00C02FF3A6DD00502D250201E86FEE
:10424000000E03012E210201E96F2A0E03012F6FD8
:1042500041DE00C02FF396DD640E0002F3CF2DF394
:10426000F4CF2EF32B0E2F6F35DE00C02FF38ADD37
:1042700000502D250201F06F000E03012E210201D6
:10428000F16F2C0E03012F6F25DE00C02FF37ADDB6
:10429000640E0002F3CF2DF3F4CF2EF32D0E2F6F0B
:1042A00019DE00C02FF36EDD00502D250201EE6FE8
:1042B000000E03012E210201EF6F04001200030122
:1042C0001251040A010ED8A4000E016E1251050A03
:1042D000010ED8A4000E006E015000120CE0566BC7
:1042E0000A0E576F880E586F000E596F090E5A6FDD
:1042F000CFEC07F00FD003011251000A0BE0566B10
:10430000030E576FA80E586F000E596F090E5A6FA3
:10431000CFEC07F004000B0E0B6E260E0C6E5D0E3C
:104320000D6E0D2EFED70C2EFCD70B2EFAD70000EB
:10433000000004000B0E0B6E260E0C6E5D0E0D6E53
:104340000D2EFED70C2EFCD70B2EFAD70000000046
:1043500004000B0E0B6E260E0C6E5D0E0D6E0D2EF8
:10436000FED70C2EFCD70B2EFAD70000000004005D
:104370000B0E0B6E260E0C6E5D0E0D6E0D2EFED707
:104380000C2EFCD70B2EFAD700000000040003010E
:104390001251040A010ED8A4000E016E1251050A32
:1043A000010ED8A4000E006E015000120CE0566BF6
:1043B0000A0E576F9E0E586F000E596F090E5A6FF6
:1043C000CFEC07F00FD003011251000A0BE0566B3F
:1043D000030E576F940E586F000E596F090E5A6FE7
:1043E000CFEC07F071EC10F0FF0E546F556B6AECD8
:1043F0000CF0FE0E0301546F556B6AEC0CF0FD0ED1
:104400000301546F556B6AEC0CF0010E0201C76F8B
:10441000010E03013D6FC0EC14F01251040A010EAD
:10442000D8A4000E016E1251050A010ED8A4000E88
:10443000006E015000120CE0566B700E576F860E26
:10444000586F000E596F010E5A6FCFEC07F00FD066
:1044500003011251000A0BE0566B080E576F660EEF
:10446000586F000E596F010E5A6FCFEC07F0FDEC3C
:104470001DF01200810E0301486F0F0E496F4A6B49
:10448000320E4B6F4C6B7CEC12F00201A251001209
:104490003FE0898E899C060E0B6E130E0C6EAD0EDE
:1044A0000D6E0D2EFED70C2EFCD70B2EFAD700006A
:1044B00000000400A251000A010ED8A4000E016EF3
:1044C00081B002D0D89001D0D880006AD8B0002A3C
:1044D0000150001605E0DCEC11F00001BD6B16D0B8
:1044E00066DC0001BD6B810E0301486F0F0E496F42
:1044F0004A6B320E4B6F4C6B7CEC12F0005204E0B6
:10450000B5EC18F00400EFD70201A26B89EC0CF0B7
:10451000810E0301486F0F0E496F020E4A6F320E73
:104520004B6F4C6B7CEC12F000524FE0040000012A
:10453000BD51000A20E1010EBD6F90C200F17AC2A8
:10454000FFF0C7C204F10201906B7A6B010EC76FD6
:104550000301566B1DEC04F090C256F3A4EC07F077
:10456000C7C23DF3C0EC14F0C3C203F10201C36B38
:1045700089EC0CF018D00001BD6B00C190F2FFC0B7
:104580007AF204C1C7F200C156F3A4EC07F07AC274
:1045900056F31DEC04F0C7C23DF3C0EC14F003C1A8
:1045A000C3F289EC0CF0810E0301486F0F0E496FC6
:1045B000020E4A6F320E4B6F4C6B7CEC12F00052C5
:1045C00004E0B5EC18F00400EED7810E0301486F4B
:1045D0000F0E496F010E4A6F320E4B6F4C6B7CEC25
:1045E00012F00001BD51000A010ED8A4000E016EA8
:1045F0000150001624E004000201C351000A03E147
:10460000010EC36F01D0C36B020E0301546FC3C20E
:1046100055F36AEC0CF089EC0CF0810E0301486F45
:104620000F0E496F010E4A6F320E4B6F4C6B7CECD4
:1046300012F0005204E0B5EC18F00400EED71200BE
:10464000810E0301486F0F0E496F4A6B320E4B6F9C
:104650004C6B7CEC12F00052D8B492D0060E0B6E6C
:10466000130E0C6EAD0E0D6E0D2EFED70C2EFCD75C
:104670000B2EFAD700000000040081A00FD0020129
:10468000C751000A03E1010EC76F01D0C76BC7C253
:104690003DF3C0EC14F089EC0CF061D05D50010AE0
:1046A00002E15D6A02D0010E5D6E5D50010A2CE1EF
:1046B00003011251040A010ED8A4000E016E12511A
:1046C000050A010ED8A4000E006E015000120CE085
:1046D000566B700E576F5B0E586F000E596F010EC0
:1046E0005A6FCFEC07F00FD003011251000A0BE014
:1046F000566B080E576F590E586F000E596F010E0A
:104700005A6FCFEC07F02BD003011251040A010EAF
:10471000D8A4000E016E1251050A010ED8A4000E95
:10472000006E015000120CE0566B700E576F3C0E7D
:10473000586F000E596F010E5A6FCFEC07F00FD073
:1047400003011251000A0BE0566B080E576F1E0E44
:10475000586F000E596F010E5A6FCFEC07F0810EA3
:104760000301486F0F0E496F4A6B320E4B6F4C6B53
:104770007CEC12F0005204E0B5EC18F00400EFD726
:10478000810E0301486F0F0E496F020E4A6F320E01
:104790004B6F4C6B7CEC12F000526DE00400030197
:1047A000810E486F0F0E496F020E4A6F320E4B6F2B
:1047B0004C6B7CEC12F000525EE0050E026E78C28B
:1047C00000F0000E016E025005E000360090013648
:1047D000FF0FFAD7010E005C026E000E0158036E47
:1047E000800E006E800E0318005C03E1025002018F
:1047F0007A5D010ED8B0000E006E5D50001607E025
:1048000002017A2B7AC256F31DEC04F02ED05D52D1
:10481000010ED8A4000E046E050E026E91C200F0C7
:10482000000E016E025005E0003600900136FF0FC9
:10483000FAD7010E005C026E000E0158036E800E66
:10484000006E800E0318005C03E102500201905DCF
:10485000010ED8B0000E006E0450001606E00201F2
:10486000902B90C256F3A4EC07F089EC0CF0B5EC59
:1048700018F0040094D7810E0301486F0F0E496FA2
:10488000010E4A6F320E4B6F4C6B7CEC12F0000144
:10489000BD51000A010ED8A4000E016E0150001691
:1048A00039E00400810E0301486F0F0E496F010EBD
:1048B0004A6F320E4B6F4C6B7CEC12F000522AE0C8
:1048C00002017A510008010ED8B0000E006E5D5052
:1048D000001606E07A077AC256F31DEC04F014D0F5
:1048E0005D52010ED8A4000E016E02019051000825
:1048F000010ED8B0000E006E0150001605E09007C2
:1049000090C256F3A4EC07F089EC0CF0B5EC18F06B
:104910000400C8D7120003012F6B6AEC1FF000C01F
:10492000F2F20050000A05E1939C939E8A8C8A8ED5
:1049300004D0938C938E8A9C8A9E1200010E0301F0
:104940002F6F6AEC1FF000C0FAF2070E2F6F6AECAF
:104950001FF000C0FBF2080E2F6F6AEC1FF000C0C2
:10496000FCF20201FA51010A03E050EC1CF060D0A5
:10497000010EF46FFD6B030E0301606FA7EC03F0F3
:104980001A0E0C6EF80E0D6E0D2EFED70C2EFCD7E7
:104990000000030E0301606FA7EC03F0060E0C6E1F
:1049A000300E0D6E0D2EFED70C2EFCD70000030E20
:1049B0000301606FA7EC03F0020E0301606FA7EC28
:1049C00003F0020E0301606FA7EC03F0080E030171
:1049D000606FA7EC03F00301606BA7EC03F0080E17
:1049E0000301606FA7EC03F00301606BA7EC03F019
:1049F000010E0301606FA7EC03F01A0E0C6EF80EA7
:104A00000D6E0D2EFED70C2EFCD700000301606B3F
:104A1000A7EC03F0060E0301606FA7EC03F003019F
:104A2000606BA7EC03F00C0E0301606FA7EC03F0C2
:104A30001200040003011251040A010ED8A4000E52
:104A4000016E1251050A010ED8A4000E006E01502D
:104A50000012D8B40AD1566B160E576F5E0E586FFF
:104A6000000E596F070E5A6FCFEC07F0020E0301CC
:104A7000566F060E576F7C0E586F000E596F090E59
:104A80005A6FCFEC07F0040E0301566F100E576FEC
:104A9000150E586F000E596F080E5A6FCFEC07F0C5
:104AA000060E0C6E300E0D6E0D2EFED70C2EFCD7A2
:104AB0000000040E0301566F100E576F150E586F4D
:104AC000000E596F080E5A6FCFEC07F0060E0C6EF1
:104AD000300E0D6E0D2EFED70C2EFCD70000040EEE
:104AE0000301566F100E576F150E586F000E596F59
:104AF000080E5A6FCFEC07F0060E0C6E300E0D6EDE
:104B00000D2EFED70C2EFCD70000060E0301566FAB
:104B1000040E576F710E586F000E596F0A0E5A6FC0
:104B2000CFEC07F004000D0E0B6E2D0E0C6ED70EA1
:104B30000D6E0D2EFED70C2EFCD70B2EFAD70000D3
:104B4000000004000B0E0B6E260E0C6E5D0E0D6E3B
:104B50000D2EFED70C2EFCD70B2EFAD7000000002E
:104B600004000301566B100E576F680E586F000E4D
:104B7000596F080E5A6FCFEC07F0020E0301566F03
:104B8000040E576FF40E586F000E596F0A0E5A6FCD
:104B9000CFEC07F0040E0301566F100E576F950E01
:104BA000586F010E596F080E5A6FCFEC07F0060EC2
:104BB0000301566F040E576F8A0E586F010E596F1E
:104BC0000A0E5A6FCFEC07F0040E0B6E0C0E0C6E33
:104BD000330E0D6E0D2EFED70C2EFCD70B2EFAD7F2
:104BE000000000000301566B100E576F810E586FC6
:104BF000010E596F080E5A6FCFEC07F0020E030139
:104C0000566F100E576FB00E586F010E596F080E89
:104C10005A6FCFEC07F0040E0301566F100E576F5A
:104C2000A70E586F010E596F080E5A6FCFEC07F0A0
:104C3000060E0301566F100E576F9E0E586F010E31
:104C4000596F080E5A6FCFEC07F00201C3530CE006
:104C50000301566B700E576F7F0E586F010E596F20
:104C6000010E5A6FCFEC07F028D103011251000A50
:104C7000D8B423D1566B040E576F5A0E586F010EDD
:104C8000596F070E5A6FCFEC07F0010E0301566FF4
:104C9000030E576F500E586F010E596F090E5A6F61
:104CA000CFEC07F004000F0E0B6E350E0C6E510E9C
:104CB0000D6E0D2EFED70C2EFCD70B2EFAD704004E
:104CC0000B0E0B6E260E0C6E5D0E0D6E0D2EFED7AE
:104CD0000C2EFCD70B2EFAD70000000004000301B5
:104CE000566B040E576F150E586F000E596F080E55
:104CF0005A6FCFEC07F0060E0C6E300E0D6E0D2EB7
:104D0000FED70C2EFCD700000301566B040E576F24
:104D1000150E586F000E596F080E5A6FCFEC07F042
:104D2000060E0C6E300E0D6E0D2EFED70C2EFCD71F
:104D300000000301566B040E576F150E586F000EDE
:104D4000596F080E5A6FCFEC07F0060E0C6E300E3E
:104D50000D6E0D2EFED70C2EFCD70000010E0301A8
:104D6000566F030E576F450E586F010E596F0A0E9E
:104D70005A6FCFEC07F004000D0E0B6E2D0E0C6E6B
:104D8000D70E0D6E0D2EFED70C2EFCD70B2EFAD79C
:104D90000000000004000B0E0B6E260E0C6E5D0E64
:104DA0000D6E0D2EFED70C2EFCD70B2EFAD7000061
:104DB000000004000301566B040E576F760E586F07
:104DC000010E596F080E5A6FCFEC07F0010E030168
:104DD000566F030E576F6B0E586F010E596F0A0E08
:104DE0005A6FCFEC07F0040E0B6E0C0E0C6E330EE8
:104DF0000D6E0D2EFED70C2EFCD70B2EFAD7000011
:104E000000000301566B576B620E586F010E596F0D
:104E1000080E5A6FCFEC07F0010E0301566F576B67
:104E2000F80E586F010E596F080E5A6FCFEC07F04D
:104E300003011251010A19E1566B090E576FF00E6A
:104E4000586F010E596F070E5A6FCFEC07F0010E25
:104E50000301566F090E576FE80E586F010E596F18
:104E6000070E5A6FCFEC07F019D00301566B090EED
:104E7000576F0C0E586F020E596F080E5A6FCFEC19
:104E800007F0010E0301566F090E576F030E586F9E
:104E9000020E596F080E5A6FCFEC07F00201C35390
:104EA0000CE00301566B080E576F010E586F020E8F
:104EB000596F010E5A6FCFEC07F0040012000FEC8F
:104EC0002BF0D0B602D0010E1D6E898C550E342405
:104ED000156E2D0E3B241C6E7AEC1FF0720E3524DD
:104EE000166E320E3A241B6E030E0B6E080E0C6EFD
:104EF000770E0D6E0D2EFED70C2EFCD70B2EFAD78B
:104F000004001E0E3624176E3B0E39241A6E90ECE8
:104F10001FF001DD420E3724186E050E0B6E0F0ECA
:104F20000C6EF10E0D6E0D2EFED70C2EFCD70B2E37
:104F3000FAD7040081B202D0028001D0029081B47D
:104F400002D0D88001D0D89002A003D002E3028022
:104F500001D0029002A003D0010E0201C06FEEDC6E
:104F600081B202D0028001D0029081B402D0D880F8
:104F700001D0D89002A003D002E3028001D00290B9
:104F800081B002D0D88001D0D89002A003D002E333
:104F9000028001D0029002A046D0030112510A0AF9
:104FA0000CE1566B030E576F2A0E586F000E596FA7
:104FB000090E5A6FCFEC07F00FD003011251000A0F
:104FC0000BE0566B0C0E576F200E586F000E596F8A
:104FD000090E5A6FCFEC07F0FF0E0301566FA4ECD9
:104FE00007F00201E451000A06E1FF0E0301566FCB
:104FF0001DEC04F004D00301566B1DEC04F0010E0F
:105000003D6FC0EC14F00B0E0B6E260E0C6E5D0E99
:105010000D6E0D2EFED70C2EFCD70B2EFAD70000EE
:1050200000000400F0D71C0E3824196E04001D5037
:10503000000A010ED8A4000E016E0201C051000A40
:10504000010ED8A4000E006E015000161DE071EC98
:1050500010F0FF0E546F556B6AEC0CF0FE0E03015E
:10506000546F556B6AEC0CF0FD0E0301546F556BD9
:105070006AEC0CF0010E0201C76F010E03013D6FD7
:10508000C0EC14F0D6DC34D01D50010A010ED8A4B7
:10509000000E016E0201C051000A010ED8A4000EDC
:1050A000006E0150001622E0FF0E03012F6F6AEC24
:1050B0001FF000C090F2FE0E2F6F6AEC1FF000C0D0
:1050C0007AF2FD0E2F6F6AEC1FF000C0C7F27AC2B1
:1050D00056F31DEC04F090C256F3A4EC07F0C7C2DF
:1050E0003DF3C0EC14F0FDEC1DF002D05FEC21F0BC
:1050F00000019351050A04E1010E0201786F0FD0FF
:1051000000019351060A04E1020E0201786F07D0F4
:1051100000019351070A03E1040E0201786F0001B8
:105120009251050A04E1010E0201916F0FD00001B6
:105130009251060A04E1020E0201916F07D00001AC
:105140009251070A03E1040E0201916F89EC0CF001
:105150000400B5EC18F00201C051000A03E13AEC7A
:1051600022F002D020EC23F0F3D7FFD70C100E0D65
:10517000120B1013006300464153542054455354FE
:1051800000464153542054455354000D07020C1B54
:1051900009121663005057523D302E3057005357B6
:1051A000523D302E303000524553455420202000CF
:1051B0006C006C00014154552D313030006C0020E2
:1051C00020202020202020004657207665722032A3
:1051D0002E350045585420626F617264006C005493
:1051E000455354204D4F44450007072020202020E0
:1051F00020202020002020202020202020200054BB
:10520000455354204D4F4445005057523D302E30A9
:1052100057002E0000433D2020202070002E00204B
:10522000005F00433D20202020704600433D2020A9
:1052300020207046005357523D302E3030005245EA
:105240005345542020200020005F002020202020F3
:1052500020202020200000002E000000433D2020C0
:1052600020307046005357523D302E30300050579A
:10527000523D302E3057002E004C3D302E303175CF
:105280004800433D2020203070004C3D302E30300F
:10529000750030433D202020307046004657207670
:1052A000657220322E350045585420626F61726459
:1052B000004154552D313030005057523D302E3082
:1052C00057002020202020202020202000202020E7
:1052D0002020202020002E005057523D302E3057E5
:1052E00000202020202020202020200020202020FE
:1052F0002020202000433D202020307046004C3DDF
:10530000302E30307548005357523D302E3030002B
:1053100054554E4500574149540054554E45004C94
:105320003D302E30307548005357523D302E3030CE
:10533000005057523D302E305700574149540043DA
:105340003D2020203070004C3D302E303075005311
:1053500057523D302E3030002E00433D202020306B
:105360007046004C3D302E30307548002020202003
:1053700020202020004F5645524C4F4144004F56AC
:1053800045524C4F4144004F5645524C4F4144000A
:10539000202020202020202000202020202020202D
:1053A00020002020202020202020004F5645524C55
:1053B0004F4144004F5645524C4F414400535752C1
:1053C0003D2020202000202020202020202000011F
:1053D00000000100005357523D20202020002020D3
:1053E00020202020202000000100102700302E3037
:1053F0003000302E303000102700202020202020C8
:105400002020002020202020202020004F56455220
:105410004C4F41440000000000000000000100FD6E
:10542000FD4C3D2020202075004C3D202020207583
:1054300048004C3D2020202075480000000000005E
:10544000000000005F00000007000700147F147FC9
:1054500014242A7F2A1223130864623649552250E5
:105460000005030000001C2241000041221C00082E
:105470002A1C2A0808083E080800503000000808C6
:10548000080808003030000020100804023E51498E
:10549000453E00427F400042615149462141454B13
:1054A000311814127F1027454545393C4A49493087
:1054B00001710905033649494936064949291E0043
:1054C000363600000056360000000814224114143D
:1054D00014141441221408000201510906324979BA
:1054E000413E7E1111117E7F494949363E4141417D
:1054F000227F4141221C7F494949417F090901011D
:105500003E414151327F0808087F00417F41002021
:1055100040413F017F081422417F404040407F02CC
:1055200004027F7F0408107F3E4141413E7F09090C
:1055300009063E4151215E7F0919294646494949DC
:105540003101017F01013F4040403F1F2040201FAB
:105550007F2018207F631408146303047804036118
:105560005149454300007F41410204081020414158
:105570007F0000040201020440404040400001025C
:10558000040020545454787F4844443838444444F8
:1055900020384444487F3854545418087E09010286
:1055A000081454543C7F0804047800447D400020D3
:1055B00040443D00007F10284400417F40007C04AF
:1055C0001804787C0804047838444444387C141463
:1055D0001408081414187C7C080404084854545413
:1055E00020043F4440203C4040207C1C2040201CA4
:1055F0003C4030403C44281028440C5050503C441F
:1056000064544C44000836410000007F0000004113
:1056100036080008082A1C08081C2A0808FF10EE93
:1056200015F0D10E006E030E016E6C0EF66E510E6B
:10563000F76E000EF86E72EC1FF01200FFFFFFFF16
:020000040030CA
:0D000100081A11FF8181FF0FC00FE00F40B2
:0200000400F00A
:100000004E01001513050001020007000700010062
:100010000050011002200450100022004500FFFF94
:100020000010002200470100022004701000FFFFB2
:10003000FFFFFFFFFFFFFFFFFFFFFFFFFFFFFFFFD0
:10004000FFFFFFFFFFFFFFFFFFFFFFFFFFFFFFFFC0
:10005000FFFFFFFFFFFFFFFFFFFFFFFFFFFFFFFFB0
:10006000FFFFFFFFFFFFFFFFFFFFFFFFFFFFFFFFA0
:10007000FFFFFFFFFFFFFFFFFFFFFFFFFFFFFFFF90
:10008000FFFFFFFFFFFFFFFFFFFFFFFFFFFFFFFF80
:10009000FFFFFFFFFFFFFFFFFFFFFFFFFFFFFFFF70
:1000A000FFFFFFFFFFFFFFFFFFFFFFFFFFFFFFFF60
:1000B000FFFFFFFFFFFFFFFFFFFFFFFFFFFFFFFF50
:1000C000FFFFFFFFFFFFFFFFFFFFFFFFFFFFFFFF40
:1000D000FFFFFFFFFFFFFFFFFFFFFFFFFFFFFFFF30
:1000E000FFFFFFFFFFFFFFFFFFFFFFFFFFFFFFFF20
:1000F000FFFFFFFFFFFFFFFFFFFFFFFFFFFFFFFF10
:00000001FF
